:1000000012C0189518951895189509C11895189546
:1000100018951895189538C018951895189518952D
:100020001895189518958FED8DBFC8EBE0EA4E2E08
:10003000DD275D2EA89584B7082E877F84BF88E1D1
:10004000992781BD91BDEEE7F0E0A0E6B0E08827FA
:100050008D933197E9F76624BE98BB9AB898BA9AFF
:10006000BC9AC298C498B69AC09878947BB77062CC
:100070007BBF70E470BD74B77F7B74BF75B77F7C46
:10008000706375BF8895F7CF0F921F922F923F92A2
:100090004F925F927F92AF92BF920F931F932F93D5
:1000A0003F934F935F936F937F938F939F93AF9300
:1000B000BF93CF93DF93EF93FF938FB78F937BB76C
:1000C0007F7D7BBF85E090E07AD0B6993BC080E031
:1000D00080936000C09A81E090E071D0B69916C01C
:1000E000B898A3E69C9197FF04C0B0990EC09F7783
:1000F0009C93B09B0AC085E09F9390E060D09F9155
:10010000B09B03C090689C933CD0E8CF0091600006
:10011000003010F009F001C015C0009160000A30F5
:1001200009F003C080E0809360007894BB9A81E876
:100130008FBD81E08EBD009160000A9384E690E05F
:1001400051D0C0987BB770627BBF8F918FBFFF91FA
:10015000EF91DF91CF91BF91AF919F918F917F915F
:100160006F915F914F913F912F911F910F91BF9090
:10017000AF907F905F904F903F902F901F900F9087
:100180001895A0E68C918F5F8C9308958E64804AB9
:100190008E4A9D4A80528E529D52805B8E5B9D5B43
:1001A00080649D64AE4AAE52AE5BAE643197F1F7A7
:1001B0000895689462F80895E89462F80895EF93BA
:1001C000FF93EE27E82BE92B31F0EDECF4E03197CB
:1001D000F1F70197D1F7FF91EF910895C895319606
:1001E000002008958F939F93442755272227332774
:1001F0000991000FECE8F1E0E00F0027F01FEEDFBF
:10020000A02CECDF902C79B7706879BF9F918F910B
:10021000D6DF79B77F7779BF88278EBD08958F9312
:100220008FB78F93EF93FF930F927F93042F152F28
:10023000490D8827581F1BD0702D022F132F2A0D10
:100240008827381F14D0602D82E0680F6695669568
:10025000061A602D88278BBD872F860F8ABD7F9158
:100260000F90FF91EF918F918FBF8F9118958FE035
:1002700018230C5F1F4F1695079516950795169531
:1002800007950F77E2E9F2E0E00F8827F81FA6DF75
:100290000895404346494C4F5255585B5E60636633
:1002A000686A6D6F7173757678797B7C7D7E7E7FF1
:1002B0007F7F7F7F7F7F7E7E7D7C7B797876757385
:1002C000716F6D6A686663605E5B5855524F4C494A
:1002D0004643403C393633302D2A2724211F1C1930
:1002E000171512100E0C0A0907060403020101007B
:1002F00000000000000001010203040607090A0CC7
:100300000E10121517191C1F2124272A2D303336E1
:02031000393C76
:00000001FF
